:2000000002C018951895479A00270BBF05BF00E009BFC29ABA9AD0E0C0E60993C036E8F313
:20002000D230D8F300E40093610000E20093630000E000936400C69ABE980FE50DBF02E014
:200040000EBFEAE9F4E029E1C8953196002D96D1D9F700E005BB0FE104BB00C0E4D1202E88
:20006000E2D1302EE0D1402E442041F0242D01D2DAD1088337FE21962A95D1F7D4D1502ECB
:20008000442061F037FE04C000916500502606C0242DEFD1099150262A95E1F752245324DB
:2000A0005424552009F04DC0022D013369F400E400936300032D003039F0013029F00230AE
:2000C00019F0033091F100C02FE60027209365000093660002E0402E75C000E90993002724
:2000E000099370C0C6D1B991A99129910991CCD12A952223D9F7F1CFBCD1B991A9912991C9
:20010000420EBAD109932A952223D9F7E6CF17D1B0D1F991E99149912AD10991CFD04A9585
:200120004423D9F704D1C29AD8CF09D1A2D1F991E9914991440E18D109934A954423D9F798
:20014000CCCF01E801C002E8222736FC0061422E302E90E8A0D0022D00936000042D0093F8
:200160006200222774C0032D0074069506950068302E00E13026229400916700040D009377
:2001800067004424552453245224022D22D1032D20D1042D1ED1052D1CD145D1202E43D130
:2001A000302E41D1402E242D3ED1088321962A95D9F739D1502E35FCD6CF00916700400E8C
:2001C00008954424002700936400022D00936000042D009362001BC00091610034FE02C0F3
:2001E00006FF0FC034FC02C006FD0BC020916400203069F000916300201B402E00E2302ED0
:200200001CC00091610010E40127009361002091640000916200402E00916300401658F0F8
:20022000401A40926200402E022F040D0093640000E2302E02C000E0302E9FEF2CD09EE140
:200240002AD000916000202E0091610030262294522C532454240DD1C20F0024D01D2F9378
:20026000242D222321F0099150262A95FACF022DB0D0032DAED0042DACD0FBD02F91C20FD9
:200280000024D01D442021F00991A3D04A94FACF052D9FD0E3CE9A95F1F7089512E01A957D
:2002A000F1F7089511E01A95F1F70895C198C09AF5DFC19AF7DF022FC098F4DF0894001FC5
:2002C00001C0000F59F0C19818F40000C09A02C0C09800C0E3DFC19AE1DFF3CFC198C09A1A
:2002E000DDDFC19AB998B898B19BFCCF8894B0990894D4DFB99AB89A089520FFDFCF331F1A
:2003000001E0C198CBDFC19AC9DF8894B0990894001FB8F7C198379510F4C09A01C0C0988B
:20032000BDDFC19ABBDFB19BFECFB8DF0895C198C098B4DFC19AB6DFC09AB0DF08953327CB
:20034000C198B99AC09AB89AC19AC298BA9A089520EAB1DF0F2FB2DF0E2FB0DF21EAA6DFDA
:200360000894CDDFE4DF0895F3DF3196089520EAA2DF0F2FA3DF0E2FA1DF089595E78BDF14
:200380002F93BE9A90E887DFC69800C000C0F02E28E0882795E77FDF00C0001FC0F0000049
:2003A000C69A00C0891F81702A95A1F795E773DF00C0879550F00000C69A00C097E76BDF5B
:2003C000C69ABE982F912A950895C698F7CFC698E9CFB69BFECF91E15EDFBE9AC69800C0CE
:2003E00000C0000028E0882794E055DF0000001FC0F00000C69A00C0891F81702A95A1F7FF
:2004000094E049DF00C0879550F00000C69A00C096E041DF000000C0C69ABE980895C698FD
:20042000F7CFC698E9CFB69BFECFB699FECF0000000096E09A95F1F701E000000000000038
:2004400000000000000000000000000095E09A95F1F786B3889486FD08940000001F68F71E
:200460000095000098E09A95F1F70000B69BFECF0895C5E6D0E00895E199FECFAEBBBFBB7B
:20048000E09A0DB311960895E199FECFAEBBBFBB0DBBE29AE19A119608953FFD9500FF9150
:1404A000817164470041532043414D204C6F61646572BB00F4
:00000001FF
